:020000040000FA
:1000000018EF1AF0C96E12000EEF16F06CEC18F033
:100010000EEC1BF0FDD7120047EF18F0D9CFE5FF2B
:10002000E1CFD9FF00C0E5FF01C0E5FF02C0E5FF59
:1000300003C0E5FF04C0E5FF05C0E5FF06C0E5FF1E
:1000400007C0E5FF08C0E5FF09C0E5FF0AC0E5FFFE
:100050000BC0E5FF0CC0E5FF0DC0E5FF0EC0E5FFDE
:100060000FC0E5FF10C0E5FF11C0E5FF12C0E5FFBE
:1000700013C0E5FF14C0E5FF15C0E5FF16C0E5FF9E
:1000800017C0E5FF18C0E5FF19C0E5FF1AC0E5FF7E
:100090001BC0E5FF1CC0E5FF1DC0E5FF1EC0E5FF5E
:1000A000020EDBCF00F0030EDBCF01F0040EDBCF3E
:1000B00002F0050EDBCF03F0060EDBCF04F0070ED7
:1000C000DBCF05F0080EDBCF06F0090EDBCF07F023
:1000D0000A0EDBCF08F0096A0A6A02C00DF00D5063
:1000E000800A0DE102500F01326F0150316F005054
:1000F000306F0F0E016E300E006E800E026E03C068
:10010000E9FF04C0F3FF055051EC1AF00B6E0B50E1
:10011000D8B4FCEF03F00B50250A02E0E3EF03F044
:100120000C6A0D6A0E6A0F6A106A0A0E116E126A64
:10013000136A146A200E156E1668176A2B0E186E55
:10014000032A02E3044A052A03C0E9FF04C0F3FFBF
:10015000055051EC1AF0196E250A13E11950E56E9D
:100160000250E56E0150E56E0050E56E73EC0FF045
:10017000040EE126094A0A2A032A02E3044A052A50
:10018000BED71950300A06E1300E156E032A02E37D
:10019000044A052A03C0E9FF04C0F3FF055051ECEF
:1001A0001AF02D0A06E1010E146E032A02E3044A36
:1001B000052A03C0E9FF04C0F3FF055051EC1AF013
:1001C000200A08E1010E176E200E186E032A02E3C2
:1001D000044A052A03C0E9FF04C0F3FF055051ECAF
:1001E0001AF02B0A06E1010E176E032A02E3044AF5
:1001F000052A03C0E9FF04C0F3FF055051EC1AF0D3
:10020000196E800F4F0F2DE31950800F460F29E212
:1002100003C019F004C01AF005C01BF019C0E9FFB3
:100220001AC0F3FF1B5051EC1AF01C6E800F500FD8
:1002300012E31C50800F460F0EE213500A0DF3CF4D
:100240001DF01D501C26D00E1C24136E192A02E32B
:100250001A4A1B2AE3D719C003F01AC004F01BC0C6
:1002600005F003C0E9FF04C0F3FF055051EC1AF09C
:100270002E0A2EE1032A02E3044A052A166A03C065
:1002800019F004C01AF005C01BF019C0E9FF1AC02C
:10029000F3FF1B5051EC1AF01C6E800F500F12E34D
:1002A0001C50800F460F0EE216500A0DF3CF1DF0C2
:1002B0001D501C26D00E1C24166E192A02E31A4A61
:1002C0001B2AE3D719C003F01AC004F01BC005F0C5
:1002D00003C0E9FF04C0F3FF055051EC1AF0196E9A
:1002E0006C0A07E1010E0C6E032A02E3044A052A98
:1002F00009D01950680A06E1010E0E6E032A02E3C6
:10030000044A052A03C0E9FF04C0F3FF055051EC7D
:100310001AF0750A06E1010E106E032A02E3044A80
:10032000052A03C0E9FF04C0F3FF055051EC1AF0A1
:10033000196E730A05E1010E0D6E200E156E3FD089
:100340001950780A03E1100E116E39D01950580A6D
:1003500005E1100E116E010E126E31D01950630AB4
:1003600002E1116A2CD019506F0A03E1080E116ED8
:1003700026D01950660A03E1010E0F6E20D01950E5
:10038000640A1DE01950690A1AE0105005E0FF0EDA
:1003900003260422052213D01950E56E0250E56EA3
:1003A0000150E56E0050E56E73EC0FF0040EE1268F
:1003B000094A0A2A032A02E3044A052AA0D60D5054
:1003C00021E00650030F0D6E000E0720196E000E7F
:1003D00008201A6E0DC006F019C007F01AC008F008
:1003E000FD0E0D26FF0E19221A220DC0E9FF19C0BD
:1003F000F3FF1A502DEC19F00D6EF3CF19F0F4CF76
:100400001AF032D10F50D8B43ED00650040F0F6E00
:10041000000E07201B6E000E08201C6E0FC006F099
:100420001BC007F01CC008F0FC0E0F26FF0E1B229D
:100430001C220FC0E9FF1BC0F3FF1C50B3EC18F0E7
:100440000F6EF3CF1BF0F4CF1CF0E9CF1DF0040EBC
:10045000196E000E0D6E800E1A6E1650E56E240E8B
:10046000E56E040EE56E000EE56E1D50E56E1C5047
:10047000E56E1B50E56E0F50E56E17EC09F0080EA7
:10048000E1261668F1D016680C5023E00650040FE0
:100490000C6E000E07200F6E000E08201B6E0CC0A5
:1004A00006F00FC007F01BC008F0FC0E0C26FF0E74
:1004B0000F221B220CC0E9FF0FC0F3FF1B50B3EC4F
:1004C00018F00C6EF3CF0FF0F4CF1BF0E9CF1CF057
:1004D0006AD00E5032E00650020F0E6E000E07205A
:1004E0001D6E000E08201E6E0EC006F01DC007F027
:1004F0001EC008F0FE0E0E26FF0E1D221E220EC08C
:10050000E9FF1DC0F3FF1E50ECEC19F00E6E0EC09B
:100510000CF0E86A0EBEFF0E0F6E1B6E1C6E1150C3
:100520000A0A03E11050D8B43ED00C500E6E0EC033
:100530000CF00F6A1B6A1C6A36D00650020F0E6E52
:10054000000E07201D6E000E08201E6E0EC006F065
:100550001DC007F01EC008F0FE0E0E26FF0E1D2265
:100560001E220EC0E9FF1DC0F3FF1E50ECEC19F077
:100570000E6EF3CF1DF00EC00CF01DC00FF0E86A38
:100580001DBEFF0E1B6E1C6E11500A0A02E11050B8
:100590000AE00C500E6E0F501D6E0EC00CF01DC008
:1005A0000FF01B6A1C6A040E196E010E0D6E800E90
:1005B0001A6E1150D8B440D0105013E01150E56EAF
:1005C000040EE56E010EE56E1C50E56E1B50E56EE7
:1005D0000F50E56E0C50E56E2BEC0BF0070EE1268C
:1005E00012D01150E56E040EE56E010EE56E1C5042
:1005F000E56E1B50E56E0F50E56E0C50E56EE9ECB4
:1006000012F0070EE12617502FE00DC0E9FF19C0C8
:10061000F3FF1A5051EC1AF02D0A26E0FF0E0D26BA
:1006200019221A2218C0E5FF0DC0E9FF19C0F3FF17
:100630001A50DDEC1AF018D00CC0E5FF0DC0E9FF30
:1006400019C0F3FF1A50DDEC1AF00D50010F0C6EBB
:10065000000E19200E6E000E1A20E56A0CC0E9FF8C
:100660000EC0F3FFDDEC1AF00DC00CF019C00EF057
:100670001AC00FF013C010F0105010E00CC0E9FFCA
:100680000EC0F3FF0F5051EC1AF0176E175006E032
:100690000C2A02E30E4A0F2A1006EED710C013F000
:1006A00014501EE109C00CF00AC00EF010C00FF08B
:1006B0000F5010E01550E56E0250E56E0150E56EEA
:1006C0000050E56E73EC0FF0040EE1260C4A0E2A82
:1006D0000F06EED70CC009F00EC00AF00FC013F0E1
:1006E00016C00CF00DC00DF019C00EF01AC00FF0BE
:1006F00009C010F00AC015F00DC0E9FF0EC0F3FFED
:100700000F5051EC1AF0166E1650D8B43ED00CC0F3
:1007100016F0176A161E171E1650171005E00CC0AB
:1007200016F00C06165031E00DC0E9FF0EC0F3FFC5
:100730000F5051EC1AF0116E125010E01150E56E8E
:10074000A9EC19F0166EE652165004E01150166E20
:10075000169A02D011C016F016C011F01150E56EB5
:100760000250E56E0150E56E0050E56E73EC0FF03F
:10077000040EE1260D2A02E30E4A0F2A104A152A1A
:100780001350D8B4B9D71306B7D710C009F015C0A5
:100790000AF014502BE010C00CF015C00DF013C07F
:1007A0000EF00E501FE0200EE56E0250E56E015077
:1007B000E56E0050E56E73EC0FF0040EE1260C4A76
:1007C0000D2A0E06EED70B50E56E0250E56E015075
:1007D000E56E0050E56E73EC0FF0040EE126094A59
:1007E0000A2A04D00CC009F00DC00AF0032A02E363
:1007F000044A052A7FEF00F00AC0F3FF0950E4CF56
:100800001EF0E4CF1DF0E4CF1CF0E4CF1BF0E4CFEA
:100810001AF0E4CF19F0E4CF18F0E4CF17F0E4CFEA
:1008200016F0E4CF15F0E4CF14F0E4CF13F0E4CFEA
:1008300012F0E4CF11F0E4CF10F0E4CF0FF0E4CFEA
:100840000EF0E4CF0DF0E4CF0CF0E4CF0BF0E4CFEA
:100850000AF0E4CF09F0E4CF08F0E4CF07F0E4CFEA
:1008600006F0E4CF05F0E4CF04F0E4CF03F0E4CFEA
:1008700002F0E4CF01F0E4CF00F0E4CFD9FF1200A2
:1008800005C0E5FF06C0E5FF07C0E5FF08C0E5FFBE
:1008900009C0E5FF0AC0E5FF0BC0E5FF0CC0E5FF9E
:1008A0000DC0E5FF0EC0E5FF0FC0E5FF10C0E5FF7E
:1008B00011C0E5FF12C0E5FF13C0E5FF14C0E5FF5E
:1008C00015C0E5FF16C0E5FF17C0E5FF18C0E5FF3E
:1008D00019C0E5FF1AC0E5FF1BC0E5FF1CC0E5FF1E
:1008E0001DC0E5FF000E00B0050F066AF60F02E31B
:1008F000062AFCD70A0F056E042E03D0FB0F01E376
:10090000062A065000B0020F00B2050F076AF60F64
:1009100002E3072AFCD70A0F066E042E03D0FB0F52
:1009200001E3072A075000B0060F00B2020F00B41F
:10093000050F086AF60F02E3082AFCD70A0F076EB4
:10094000042E03D0FB0F01E3082A085000B2010F68
:1009500000B4020F00B6050F096AF60F02E3092A78
:10096000FCD70A0F086E042E03D0FB0F01E3092AFF
:10097000095000B0090F00B2080F00B4060F00B60E
:10098000020F00B8050F0A6AF60F02E30A2AFCD725
:100990000A0F096E042E03D0FB0F01E30A2A0A5046
:1009A00000B0030F00B2070F00B4050F00B6010F2F
:1009B00000B8020F00BA050F0B6AF60F02E30B2A0C
:1009C000FCD70A0F0A6E042E03D0FB0F01E30B2A9B
:1009D0000B5000B0050F00B4010F00B6030F00B8B4
:1009E000060F00BA020F00BC050F0C6AF60F02E3F7
:1009F0000C2AFCD70A0F0B6E042E03D0FB0F01E369
:100A00000C2A0C5000B0070F00B2050F00BA010FFE
:100A100000BC020F00BE050F0D6AF60F02E30D2A9F
:100A2000FCD70A0F0C6E042E03D0FB0F01E30D2A36
:100A30000D5000B0070F00B2050F00B4010F00B653
:100A4000020F00B8040F00BA080F00BC060F00BE6A
:100A5000020F01B0050F0E6AF60F02E30E2AFCD753
:100A60000A0F0D6E042E03D0FB0F01E30E2A0E5069
:100A700000B0040F00B2090F00B4090F00B6080F50
:100A800000B8060F00BA020F00BC050F00BE010F30
:100A900001B0020F01B2050F0F6AF60F02E30F2A31
:100AA000FCD70A0F0E6E042E03D0FB0F01E30F2AB2
:100AB0000F5000B0040F00B2080F00B4070F00B6CB
:100AC000050F00B8010F00BA030F00BC060F00BEEF
:100AD000030F01B0060F01B2020F01B4050F106A37
:100AE000F60F02E3102AFCD70A0F0F6E042E03D074
:100AF000FB0F01E3102A105000B0060F00B2020FE6
:100B000000B4050F00B6010F00B8030F00BA060FBE
:100B100000BC020F00BE050F01B2010F01B4020FAD
:100B200001B6050F116AF60F02E3112AFCD70A0F6E
:100B3000106E042E03D0FB0F01E3112A115000B0F8
:100B4000040F00B2090F00B4080F00B6070F00B879
:100B5000040F00BA080F00BC070F00BE040F01B05D
:100B6000090F01B2080F01B4060F01B6020F01B858
:100B7000050F126AF60F02E3122AFCD70A0F116E54
:100B8000042E03D0FB0F01E3122A125000B4010F10
:100B900000B6030F00B8070F00BA040F00BC090F1E
:100BA00000BE090F01B0080F01B2070F01B4050F15
:100BB00001B6010F01B8020F01BA050F136AF60F53
:100BC00002E3132AFCD70A0F126E042E03D0FB0F88
:100BD00001E3132A135000B0060F00B2020F00B455
:100BE000040F00B6080F00B8060F00BA030F00BCD0
:100BF000060F00BE030F01B0070F01B2050F01B4CD
:100C0000010F01B6030F01B8060F01BA020F01BCB4
:100C1000050F146AF60F02E3142AFCD70A0F136EAD
:100C2000042E03D0FB0F01E3142A145000B0090F67
:100C300000B2090F00B4080F00B6060F00B8030F8A
:100C400000BA070F00BC040F00BE090F01B0080F67
:100C500001B2070F01B4050F01BA010F01BC020F69
:100C600001BE050F156AF60F02E3152AFCD70A0F1D
:100C7000146E042E03D0FB0F01E3152A155000B0AB
:100C8000050F00B2010F00B4030F00B6070F00B844
:100C9000050F00BC010F00BE020F01B0050F01B22D
:100CA000010F01B4030F01B6070F01B8040F01BA19
:100CB000080F01BC060F01BE020F02B0050F166A35
:100CC000F60F02E3162AFCD70A0F156E042E03D086
:100CD000FB0F01E3162A165000B2010F00B4020FF9
:100CE00000B6040F00B8090F00BA090F00BC080FC6
:100CF00000BE060F01B0020F01B2050F01B8010FCF
:100D000001BA020F01BC050F01BE010F02B0020FB4
:100D100002B2050F176AF60F02E3172AFCD70A0F73
:100D2000166E042E03D0FB0F01E3172A175000BAEA
:100D3000010F00BC030F00BE070F01B0050F01B487
:100D4000010F01B6020F01B8040F01BA080F01BC70
:100D5000060F01BE030F02B0060F02B2020F02B46B
:100D6000050F186AF60F02E3182AFCD70A0F176E50
:100D7000042E03D0FB0F01E3182A185001B0010F15
:100D800001B2030F01B4060F01B6020F01B8040F40
:100D900001BA080F01BC070F01BE050F02B2010F17
:100DA00002B4020F02B6050F196AF60F02E3192A00
:100DB000FCD70A0F186E042E03D0FB0F01E3192A8B
:100DC000195001B6010F01B8020F01BA040F01BC9E
:100DD000090F01BE090F02B0090F02B2080F02B4D9
:100DE000060F02B6020F02B8050F1A6AF60F02E3E9
:100DF0001A2AFCD70A0F196E042E03D0FB0F01E349
:100E00001A2A1A5001BE010F02B0030F02B2070FD7
:100E100002B4050F02B6010F02B8020F02BA050FA5
:100E20001B6AF60F02E31B2AFCD70A0F1A6E042E68
:100E300003D0FB0F01E31B2A1B5002B4010F02B6C3
:100E4000030F02B8060F02BA020F02BC050F1C6A9C
:100E5000F60F02E31C2AFCD70A0F1B6E042E03D0E8
:100E6000FB0F01E31C2A1C5002BA010F02BC020F47
:100E700002BE050F1D6AF60F02E31D2AFCD70A0FFA
:100E80001C6E042E03D0FB0F01E31D2A300FEE6E03
:100E90001B50300FEE6E1A50300FEE6E1950300F9F
:100EA000EE6E1850300FEE6E1750300FEE6E16507B
:100EB000300FEE6E1550300FEE6E1450300FEE6E98
:100EC0001350300FEE6E1250300FEE6E1150300F87
:100ED000EE6E1050300FEE6E0F50300FEE6E0E5063
:100EE000300FEE6E0D50300FEE6E0C50300FEE6E78
:100EF0000B50300FEE6E0A50300FEE6E0950300F6F
:100F0000EE6E0850300FEE6E0750300FEE6E06504A
:100F1000300FEE6E0550300FEE6E170EE4CF1DF061
:100F2000E4CF1CF0E4CF1BF0E4CF1AF0E4CF19F0CB
:100F3000E4CF18F0E4CF17F0E4CF16F0E4CF15F0CB
:100F4000E4CF14F0E4CF13F0E4CF12F0E4CF11F0CB
:100F5000E4CF10F0E4CF0FF0E4CF0EF0E4CF0DF0CB
:100F6000E4CF0CF0E4CF0BF0E4CF0AF0E4CF09F0CB
:100F7000E4CF08F0E4CF07F0E4CF06F0E4CF05F0CB
:100F8000120000C0E5FF01C0E5FF02C0E5FF03C09D
:100F9000E5FF04C0E5FF05C0E5FF06C0E5FF07C0AB
:100FA000E5FF08C0E5FF09C0E5FF0AC0E5FF0BC08B
:100FB000E5FF0CC0E5FF0DC0E5FF0EC0E5FF000E2C
:100FC00000B0010F00B2020F00B4040F00B6080F0A
:100FD00000B8060F00BA020F00BC040F00BE080FD5
:100FE00001B0060F01B2020F01B4040F01B6080FE1
:100FF00001B8060F01BA020F01BC040F01BE080FB1
:1010000002B0060F02B2020F02B4040F02B6080FBC
:1010100002B8060F02BA020F02BC040F02BE080F8C
:10102000056AF60F02E3052AFCD70A0F046E055085
:1010300000B8010F00BA030F00BC060F00BE020F7C
:1010400001B0050F01B2010F01B4020F01B6040F88
:1010500001B8090F01BA090F01BC080F01BE060F44
:1010600002B0030F02B2070F02B4040F02B6080F5A
:1010700002B8070F02BA050F066AF60F02E3062A46
:10108000FCD70A0F056E065000BE010F01B0020F1B
:1010900001B2050F01BA010F01BC030F01BE070F1A
:1010A00002B0050F02B4010F02B6020F02B8050F1D
:1010B00002BA010F02BC030F02BE060F076AF60F49
:1010C00002E3072AFCD70A0F066E075001B4010F8E
:1010D00001B6020F01B8040F01BA080F01BC060FD8
:1010E00001BE020F02B0050F02B2010F02B4020FDF
:1010F00002B6040F02B8080F02BA070F02BC040FB1
:1011000002BE080F086AF60F02E3082AFCD70A0F8E
:10111000076E085001BC010F01BE030F02B0060F9D
:1011200002B2030F02B4060F02B6020F02B8040F98
:1011300002BA090F02BC090F02BE080F096AF60FB6
:1011400002E3092AFCD70A0F086E095002B2010F08
:1011500002B4020F02B6050F02BC010F02BE030F5C
:101160000A6AF60F02E30A2AFCD70A0F096E0A5030
:1011700002B8010F02BA020F02BC040F02BE080F30
:101180000B6AF60F02E30B2AFCD70A0F0A6E0B500C
:101190000E6A0EE10A5010E1095012E1085014E104
:1011A000075016E1065018E105501AE104501CD012
:1011B0000E2A300FEE6E0A500E2A300FEE6E0950D6
:1011C0000E2A300FEE6E08500E2A300FEE6E0750CA
:1011D0000E2A300FEE6E06500E2A300FEE6E0550BE
:1011E0000E2A300FEE6E04500E2A300FEE6E0E50A7
:1011F000E4CF0EF0E4CF0DF0E4CF0CF0E4CF0BF031
:10120000E4CF0AF0E4CF09F0E4CF08F0E4CF07F030
:10121000E4CF06F0E4CF05F0E4CF04F0E4CF03F030
:10122000E4CF02F0E4CF01F0E4CF00F01200D9CF18
:10123000E5FFE1CFD9FF00C0E5FF01C0E5FF02C037
:10124000E5FF03C0E5FF04C0E5FF05C0E5FF06C0FC
:10125000E5FF07C0E5FF08C0E5FF09C0E5FF0AC0DC
:10126000E5FF0BC0E5FF020EDBCF00F0030EDBCF86
:1012700001F0040EDBCF02F0050EDBCF03F0060E0B
:10128000DBCF04F0070EDBCF05F0080EDBCF06F056
:10129000090EDBCF07F006C008F0060608500EE086
:1012A00006500424086EE86A06BEE8680520096E48
:1012B00008C0E9FF09C0EAFFEF6AEDD700500F014F
:1012C000236F0150246F0250256F0350266F23CFE8
:1012D00000F024CF01F025CF02F026CF03F0066AFC
:1012E000086A096A800E03140A6E065007E1085066
:1012F00005E1095003E10A50800A01E012D0039E83
:1013000000500F01236F0150246F0250256F0350CE
:10131000266F04C0E9FF05C0EAFF2D0EEF6E044AF8
:10132000052A0F01253526357E08006E2351016EF2
:101330002451026E7F0E2515036E066A038E086A1D
:10134000096A0A6A0B6A005019E0D88000AED8908A
:101350000EE30850082609360A360B3603BE08800D
:1013600001500126023603360636002AECD7D89003
:1013700006320332023201320006E5D70850091066
:101380000A100B1012E00550E56E0450E56E0B508C
:10139000E56E0A50E56E0950E56E0850E56E7BEC8F
:1013A00017F0006E060EE12608D004C0E9FF05C064
:1013B000EAFF300EEF6E010E006E00500426E86A60
:1013C00000BEE8680522075028E004C0E9FF05C018
:1013D000EAFF2E0EEF6E002A044A052A075018086D
:1013E000E56E0550E56E0450E56E0650E56E03505F
:1013F000E56E0250E56E0150E56EE8EC16F0016E08
:10140000070EE1260150002607500426E86A05224F
:1014100004C0E9FF05C0EAFFEF6A0050E4CF0BF01B
:10142000E4CF0AF0E4CF09F0E4CF08F0E4CF07F00E
:10143000E4CF06F0E4CF05F0E4CF04F0E4CF03F00E
:10144000E4CF02F0E4CF01F0E4CF00F0E4CFD9FF25
:10145000120000C0E5FF01C0E5FF04017951D8B4D6
:10146000F5D09DA81DD09EA81BD004019951040160
:10147000961905E190EC1AF00401966BE7D0000E86
:1014800004019925006E016A0F0E012200C0E9FFD8
:1014900001C0EAFFEFCF36FF992B36CFADFFD6D094
:1014A0009EAAD4D0ABA205D00401978190EC1AF08B
:1014B000CDD0ABA405D00401978390EC1AF0C6D030
:1014C000ABA03ED0AECF36FF800E04017A110F01E3
:1014D000361904E104019789AB96B8D00F01365153
:1014E00004E0365104017A1927E104019799AB967B
:1014F0000F01365103E00401979702D0040197874A
:1015000036CF9BF494C49CF40401940504019D6FB0
:10151000600E04019C25006E016A000E012200C0CD
:10152000E9FF01C0EAFF36CFEFFF9C2B9C51800AF8
:1015300002E104019C6B8AD004019799AB8686D0A6
:10154000AECF36FF040197A919D0800E04017A119D
:101550000F01361911E18B909D9AAB9804019651B9
:1015600004E1AD6A90EC1AF007D000CFADFF010E98
:101570000401996F9D886AD0AB8668D00F013651FF
:1015800004019B2704019C5104019D191BE10401E6
:101590009B510CE19CC494F4040197B712D08B903A
:1015A0009D9AAB98AD6A90EC1AF00BD00401978528
:1015B00097B707D08B909D9AAB98010EAD6E90ECCB
:1015C0001AF044D004019C510401951908E104016A
:1015D00095510401941903E090EC1AF037D094C4AB
:1015E00000F0016A004A012AE56A800EE56E0150AA
:1015F000E56E0050E56E77EC10F0006E040EE1260B
:1016000000500401936F04019C190CE11F0E0F019F
:10161000361504019D6F9D2B9D2B040194510401EF
:101620009D279D9F9CC400F004019C2B016A600EC5
:101630000026000E012200C0E9FF01C0EAFF36CFFC
:10164000EFFF9C51800A02E104019C6BE4CF01F0A2
:10165000E4CF00F01200D9CFE5FFE1CFD9FF00C001
:10166000E5FF01C0E5FF02C0E5FF03C0E5FF04C0E0
:10167000E5FF05C0E5FF06C0E5FF07C0E5FF08C0C0
:10168000E5FF09C0E5FF0AC0E5FF0BC0E5FF0CC0A0
:10169000E5FF0DC0E5FF0EC0E5FF0FC0E5FF020E40
:1016A000DBCF00F0030EDBCF01F0040EDBCF02F046
:1016B000050EDBCF03F0060EDBCF04F0070EDBCF09
:1016C00005F0080EDBCF06F0200E076E086A06C094
:1016D00009F00A6A0B6A0C6AE56AE56AE56A09506C
:1016E000E56E0350E56E0250E56E0150E56E005068
:1016F000E56EB4EC0CF00D6E080EE126300E0D26F2
:101700003A0E0D5C05E30D500E6E270E0E240D6E85
:10171000FF0E07260822E00E07240E6E000E08209A
:101720000F6E0EC0E9FF0FC0EAFF0DC0EFFF0C50B7
:10173000E56E0B50E56E0A50E56E0950E56E0350FC
:10174000E56E0250E56E0150E56E0050E56ED4EC9A
:101750000DF0006EF3CF01F0F4CF02F0E9CF03F00B
:10176000080EE1260050011002100310D8A4AFD7D4
:1017700007C000F008C001F004C002F005C003F08B
:1017800000C004F001C005F0004A012AE00E042662
:10179000000E052204C0E9FF05C0EAFFEFCF04F008
:1017A00002C0E9FF03C0EAFF04C0EFFF024A032AB8
:1017B000000E015C02E1200E005CE2E302C0E9FFE2
:1017C00003C0EAFF000EEF6AE4CF0FF0E4CF0EF0A3
:1017D000E4CF0DF0E4CF0CF0E4CF0BF0E4CF0AF04F
:1017E000E4CF09F0E4CF08F0E4CF07F0E4CF06F04F
:1017F000E4CF05F0E4CF04F0E4CF03F0E4CF02F04F
:10180000E4CF01F0E4CF00F0E4CFD9FF120000C034
:10181000E5FF01C0E5FF02C0E5FF03C0E5FFA6EC60
:1018200017F0006EF3CF01F0F4CF02F0E9CF03F030
:1018300004018E51005E8F51015A9051025A91510C
:10184000035A039E3F0E035C08E1FF0E025C05E1B4
:10185000FF0E015C02E1FF0E005C16E230EC1BF0B3
:10186000A6EC17F0F3CF01F0F4CF02F0E9CF03F0CC
:10187000500F04018E6F460E01208F6F000E022064
:10188000906F000E0320916F080E04017C5DD8B0AC
:1018900062D00F014EB15FD004017C51020DF450B3
:1018A000016EF3CF00F0240E0026040E012200C0CA
:1018B000E9FF01C0EAFFEECF02F0EFCF03F00250E4
:1018C000031002E17C2B47D004017C51030DF4503E
:1018D000036EF3CF02F05C0E0226040E032202C058
:1018E000E9FF03C0EAFFEECF27FFEECF28FFEFCFDF
:1018F00029FF810E7C25026E036A040E032202C0BA
:10190000E9FF03C0EAFFEFCFA1F400C0E9FF01C087
:10191000EAFFEECF00F0EFCF01F0001E011E0150F4
:101920000F01506F00500F014F6F7E9204C0E5FF12
:10193000F2CF04F0F29E0F012751E96E2851EA6EB2
:101940000401A151EF120F014E8104BEF28EE4CFCB
:1019500004F004017C2BE4CF03F0E4CF02F0E4CFE9
:1019600001F0E4CF00F01200D9CFE5FFE1CFD9FFBD
:1019700000C0E5FF01C0E5FF02C0E5FF03C0E5FFD1
:1019800004C0E5FF05C0E5FF06C0E5FF07C0E5FFB1
:1019900008C0E5FF09C0E5FF0AC0E5FF020EDBCF86
:1019A00000F0030EDBCF01F0040EDBCF02F0050EDA
:1019B000DBCF03F0060EDBCF04F0070EDBCF05F024
:1019C000080EDBCF06F0090EDBCF07F0086A096AC4
:1019D0000750800BE8440A6E0A501BE104500426AD
:1019E0000536063607360750035C08E10650025CF0
:1019F00005E10550015C02E10450005C06E2D8906C
:101A0000073206320532043204D0092A09C008F030
:101A1000DFD70750035C08E10650025C05E1055082
:101A2000015C02E10450005C08E30450005E0550D4
:101A3000015A0650025A0750035AD890073206320C
:101A40000532043208C009F008060950E2E103C07B
:101A5000E9FF02C0F4FF01C0F3FF0050E4CF0AF039
:101A6000E4CF09F0E4CF08F0E4CF07F0E4CF06F0CC
:101A7000E4CF05F0E4CF04F0E4CF03F0E4CF02F0CC
:101A8000E4CF01F0E4CF00F0E4CFD9FF120000C0B2
:101A9000E5FF01C0E5FF03C0E5FF04C0E5FF05C0A9
:101AA000E5FF06C0E5FF07C0E5FF08C0E5FF09C088
:101AB000E5FF0AC0E5FF0BC0E5FF7EC400F07FC470
:101AC00001F004017E3F01D07F2B0050E56E82ECD7
:101AD0001AF0E652076E046A056A066A7EC400F0D0
:101AE0007FC401F004017E3F01D07F2B0050E56EE2
:101AF00082EC1AF0E6520B6A0A6E086A0850041269
:101B000005120A5006120B5007127EC400F07FC463
:101B100001F004017E3F01D07F2B0050E56E82EC86
:101B20001AF0E652036E006A03C001F0E86A03BED1
:101B3000FF0E086E096E0050041201500512085085
:101B40000612095007127EC400F07FC401F00401A0
:101B50007E3F01D07F2B0050E56E82EC1AF0E652FA
:101B6000016A0412015005120612071207C0E9FFAC
:101B700006C0F4FF05C0F3FF0450E4CF0BF0E4CF40
:101B80000AF0E4CF09F0E4CF08F0E4CF07F0E4CFA7
:101B900006F0E4CF05F0E4CF04F0E4CF03F0E4CFA7
:101BA00001F0E4CF00F01200D9CFE5FFE1CFD9FF7B
:101BB00000C0E5FF01C0E5FF02C0E5FF03C0E5FF8F
:101BC00004C0E5FF05C0E5FF06C0E5FF07C0E5FF6F
:101BD00008C0E5FF09C0E5FF0AC0E5FF0BC0E5FF4F
:101BE0000CC0E5FF0DC0E5FF020EDBCF00F0030ED9
:101BF000DBCF01F0040EDBCF02F0050EDBCF03F0EC
:101C0000060EDBCF04F0070EDBCF05F0080EDBCFAE
:101C100006F0090EDBCF07F0086A096A0A6A0B6A48
:101C2000200E0C6E0350800BE8440D6E0050002611
:101C30000136023603360850082609360A360B36B6
:101C40000D50D8A4088007500B5C08E106500A5CD0
:101C500005E10550095C02E10450085C09E3045009
:101C6000085E0550095A06500A5A07500B5A008060
:101C70000C2ED8D703C0E9FF02C0F4FF01C0F3FF68
:101C80000050E4CF0DF0E4CF0CF0E4CF0BF0E4CF44
:101C90000AF0E4CF09F0E4CF08F0E4CF07F0E4CF96
:101CA00006F0E4CF05F0E4CF04F0E4CF03F0E4CF96
:101CB00002F0E4CF01F0E4CF00F0E4CFD9FF12004E
:101CC00000C0E5FF01C0E5FF02C0E5FF03C0E5FF7E
:101CD00004C0E5FF040195510401941901E15CD0B1
:101CE00095C400F0002A009E600E0024016E026A76
:101CF000000E022201C0E9FF02C0EAFFEFCF9FF40D
:101D00001F0E04019F1795C49EF49F5104019E2746
:101D10009E2B9E2B9E9FD0EC17F0016E015003E18D
:101D2000016A012A01D0016AD0EC17F004019F6F0B
:101D3000800E9F15026E1F0E9F15036E03C004F0E8
:101D400003C09FF4045003E194C495F438D00150CB
:101D50001BE002501FE0D0EC17F0006E04019F075B
:101D60000050420A17E000504E0A03E199EC14F0CB
:101D700011D00050460A03E1D2EC1AF00BD000500B
:101D8000490A08E1FF0006D095C4A0F40250D8B477
:101D9000F9EC1AF09EC495F4040176510401771908
:101DA00006E00401965103E1EAEC0EF008D08BB096
:101DB00006D00401965103E1ACB290EC1AF0E4CFE6
:101DC00004F0E4CF03F0E4CF02F0E4CF01F0E4CF7D
:101DD00000F0120000C0E5FF01C0E5FF02C0E5FF12
:101DE00003C0E5FFACA276D0D3EC18F0006E005033
:101DF00005E10401776B0401766B6CD077C401F0C8
:101E000000500126D3EC18F0026E00060250230A9F
:101E10001FE1010E005CD8A05BD0D3EC18F0026E7D
:101E2000690A03E14BEC17F053D00250720A03E148
:101E300090EC1AF04DD00250730A01E049D08B802B
:101E4000AB869D8A9D98AE50AE50AB98AB8840D083
:101E50000250430A05E00250420A01E039D001D0A5
:101E6000008E00C098F400500F01006F010E0401B5
:101E7000996F04017751011814E0D3EC18F0026E49
:101E800004019827000E04019925006E036A0F0EC5
:101E9000032200C0E9FF03C0EAFF02C0EFFF992B55
:101EA000E8D7000E04019925006E026A0F0E022287
:101EB0000401981D036E032A00C0E9FF02C0EAFF77
:101EC00003C0EFFF0401992B99C496F40F01346B02
:101ED00001C077F4E4CF03F0E4CF02F0E4CF01F0E7
:101EE000E4CF00F01200D9CFE5FFE1CFD9FF00C069
:101EF000E5FF01C0E5FF02C0E5FF03C0E5FF04C048
:101F0000E5FF05C0E5FF06C0E5FF07C0E5FF020EDF
:101F1000DBCF00F0030EDBCF01F0040EDBCF02F0CD
:101F2000050EDBCF03F002C006F00650046E800AF7
:101F300033E100C0E9FF01C0F3FF02502DEC19F0BE
:101F4000056EF3CF06F0F4CF07F003C0E5FF05C040
:101F5000E9FF06C0F3FF0750DDEC1AF000C0E9FF0F
:101F600001C0F3FF02502DEC19F0056EF3CF06F01F
:101F7000F4CF07F0052A02E3064A072A05C0E5FF69
:101F800006C0F4FF07C0F6FF00C0E9FF01C0F3FF81
:101F9000025073EC1AF01DD004AA1BD0047A04502E
:101FA00004E103501DEC1BF014D00450010A04E1BD
:101FB000035002EC00F00DD004500F0A04E103506E
:101FC0001AEC17F006D004500E0A03E1035033EC6C
:101FD0001BF0E4CF07F0E4CF06F0E4CF05F0E4CF48
:101FE00004F0E4CF03F0E4CF02F0E4CF01F0E4CF5B
:101FF00000F0E4CFD9FF1200D9CFE5FFE1CFD9FF40
:1020000000C0E5FF01C0E5FF02C0E5FF03C0E5FF3A
:1020100004C0E5FF05C0E5FF06C0E5FF07C0E5FF1A
:10202000020EDBCF00F0030EDBCF01F0040EDBCF9E
:1020300002F0050EDBCF03F077C478F4040176518B
:102040000401785F780703C004F0056A030E0426D4
:10205000D8B0052A78C406F0076A0750800FF36EDF
:102060000550800FF35C02E10450065C02E2E86870
:102070002BD0020E035C02E2E86A26D0030603506E
:10208000E56E97EC15F0E652046A0350045C14E226
:1020900004500024056EE86A0120066EE86A0220FA
:1020A00005C0E9FF06C0F3FF51EC1AF0042AE56E03
:1020B00097EC15F0E652E9D777C478F4040176512D
:1020C0000401785F7807E86AE4CF07F0E4CF06F010
:1020D000E4CF05F0E4CF04F0E4CF03F0E4CF02F066
:1020E000E4CF01F0E4CF00F0E4CFD9FF1200D9CF64
:1020F000E5FFE1CFD9FF00C0E5FF01C0E5FF02C069
:10210000E5FF03C0E5FF04C0E5FF05C0E5FF06C02D
:10211000E5FF020EDBCF00F0030EDBCF01F0040E73
:10212000DBCF02F0050EDBCF03F0D88001AED890F4
:10213000046A0436045007E0011C066E001C056E9C
:10214000054A062A04D000C005F001C006F0D88078
:1021500003AED89007E3031C016E021C006E004A18
:10216000012A04D002C000F003C001F00150E56E66
:102170000050E56E0650E56E0550E56E4CEC13F030
:10218000006EF3CF01F0040EE12604500AE0011CBA
:10219000036E001C026E024A032A03C0F3FF0250C2
:1021A00003D001C0F3FF0050E4CF06F0E4CF05F008
:1021B000E4CF04F0E4CF03F0E4CF02F0E4CF01F089
:1021C000E4CF00F0E4CFD9FF1200D9CFE5FFE1CF93
:1021D000D9FF00C0E5FF01C0E5FF02C0E5FF03C075
:1021E000E5FF04C0E5FF05C0E5FF020EDBCF00F010
:1021F000030EDBCF01F0040EDBCF02F0050EDBCFC8
:1022000003F07EC404F07FC405F004017E3F01D0DA
:102210007F2B0350E56E0450E56EFAEC17F0E652A2
:10222000E6527EC404F07FC405F004017E3F01D075
:102230007F2B0250056EE56E0450E56EFAEC17F048
:10224000E652E6527EC404F07FC405F004017E3FEE
:1022500001D07F2B0150056EE56E0450E56EFAEC5F
:1022600017F0E652E6527EC404F07FC405F0040184
:102270007E3F01D07F2B0050E56E0450E56EFAECF6
:1022800017F0E652E652E4CF05F0E4CF04F0E4CFD5
:1022900003F0E4CF02F0E4CF01F0E4CF00F0E4CFAC
:1022A000D9FF120000C0E5FF01C0E5FF02C0E5FF55
:1022B00003C0E5FF04C0E5FF05C0E5FF06C0E5FF7C
:1022C0000F014E6B0F014E894E837D827F82006A23
:1022D000016A026A036A046A5C0E0124056E040E38
:1022E0000220066E05C0E9FF06C0EAFFEE6AEE6A4C
:1022F000EF6A240E0324056E040E0420066E05C04A
:10230000E9FF06C0EAFFEE6AEF6A030E0126D8B0C5
:10231000022A020E0326D8B0042A002A080E005C06
:10232000DBE304017C6BA6EC17F0F3CF01F0F4CFF4
:1023300002F0E9CF03F0500F04018E6F460E01202A
:102340008F6F000E0220906F000E0320916FE4CF7C
:1023500006F0E4CF05F0E4CF04F0E4CF03F0E4CFDF
:1023600002F0E4CF01F0E4CF00F012002564202554
:10237000640A0000D9CFE5FFE1CFD9FF00C0E5FF37
:1023800001C0E5FF02C0E5FF03C0E5FF04C0E5FFB3
:1023900005C0E5FF06C0E5FF020EDBCF00F0030E2F
:1023A000DBCF01F0040EDBCF02F00F01335119E156
:1023B00047EC0DF0036EF3CF04F0F4CF05F0E9CF56
:1023C00006F003C0E5FF04C0F4FF05C0F6FF06C039
:1023D000F7FF00C0E9FF01C0F3FF025062EC1AF002
:1023E0001ED00F013351010A1AE100C0E9FF01C0FC
:1023F000F3FF0250B3EC18F0006EF3CF01F0F4CF0E
:1024000002F0E9CF03F00350E56E0250E56E015093
:10241000E56E0050E56EE5EC10F0040EE126E4CF29
:1024200006F0E4CF05F0E4CF04F0E4CF03F0E4CF0E
:1024300002F0E4CF01F0E4CF00F0E4CFD9FF1200C6
:1024400000C0E5FF01C0E5FF02C0E5FF03C0E5FFF6
:1024500004C0E5FFD0EC17F0006EFE0A2DE1A9ECF8
:1024600013F0D0EC17F0016E080E015CD8B043D029
:102470000150020DF450036EF3CF02F0240E022639
:10248000040E032202C0E9FF03C0EAFFEECF02F010
:10249000EFCF03F00350E56E0250E56EE56A0150A0
:1024A000E56E000EE56E230EE56E6C0EE56EDBEC60
:1024B00014F0070EE1261FD0080E005C1CE2D0ECE1
:1024C00017F0046E036AD0EC17F0026A032602507C
:1024D00004220050020DF450016EF3CF00F0240EE0
:1024E0000026040E012200C0E9FF01C0EAFF03C07C
:1024F000EEFF04C0EFFFE4CF04F0E4CF03F0E4CF3D
:1025000002F0E4CF01F0E4CF00F01200D9CFE5FFF4
:10251000E1CFD9FF00C0E5FF01C0E5FF02C0E5FF44
:1025200003C0E5FF04C0E5FF05C0E5FF06C0E5FF09
:10253000020EDBCF00F0030EDBCF01F0040EDBCF89
:1025400002F0050EDBCF03F0060EDBCF04F00050E7
:10255000030DF450066EF3CF05F05C0E0526040E55
:10256000062205C0E9FF06C0EAFF01C0EEFF02C077
:10257000EEFF03C0EFFF810E0024016E026A040E1D
:10258000022201C0E9FF02C0EAFF04C0EFFF0050D1
:10259000020DF450016EF3CF00F0240E0026040E5D
:1025A000012200C0E9FF01C0EAFF000EEE6AEF6AF7
:1025B000E4CF06F0E4CF05F0E4CF04F0E4CF03F07D
:1025C000E4CF02F0E4CF01F0E4CF00F0E4CFD9FF94
:1025D0001200D9CFE5FFE1CFD9FF00C0E5FF01C070
:1025E000E5FF02C0E5FF03C0E5FF04C0E5FF05C04D
:1025F000E5FF06C0E5FF020EDBCF00F0030EDBCFE8
:1026000001F0040EDBCF02F0050EDBCF03F0060E67
:10261000DBCF04F0070EDBCF05F0080EDBCF06F0B2
:10262000D88003AED89015E306500A0A12E104C020
:10263000E9FF05C0EAFF2D0EEF6E044A052A031ECE
:10264000021E011E006C05E1012A03E1022AD8B432
:10265000032A0650E56E0550E56E0450E56E035002
:10266000E56E0250E56E0150E56E0050E56E2BEC14
:102670000BF0070EE126E4CF06F0E4CF05F0E4CF3F
:1026800004F0E4CF03F0E4CF02F0E4CF01F0E4CFB4
:1026900000F0E4CFD9FF1200D9CFE5FFE1CFD9FF99
:1026A00000C0E5FF01C0E5FF02C0E5FF03C0E5FF94
:1026B00004C0E5FF05C0E5FF06C0E5FF020EDBCF65
:1026C00000F0030EDBCF01F0040EDBCF02F0050EAD
:1026D000DBCF03F0046A056A0350800BE844066E02
:1026E000065011E10250022603360350015C02E15C
:1026F0000250005C04E2D8900332023204D0052A72
:1027000005C004F0E9D70350015C02E10250005C0F
:1027100004E30250005E0350015AD89003320232A3
:1027200004C005F004060550EEE101C0F3FF0050BF
:10273000E4CF06F0E4CF05F0E4CF04F0E4CF03F0FB
:10274000E4CF02F0E4CF01F0E4CF00F0E4CFD9FF12
:10275000120000C0E5FF01C0E5FF02C0E5FF03C0B5
:10276000E5FF95C400F0016AA0C402F0036A0250BC
:10277000005E0350015AE56A800EE56E0150E56E79
:102780000050E56E77EC10F0006E040EE1260006B6
:10279000A0C401F0430E1AEC17F0200E1AEC17F04B
:1027A0000050800F7F0F20E3600E0124026E036A49
:1027B000000E032202C0E9FF03C0EAFFEFCF02F0E0
:1027C000E56A0250E56E000EE56E350EE56E380ED8
:1027D000E56EDBEC14F0050EE126012A0150800ABB
:1027E00001E1016A0006DCD7E4CF03F0E4CF02F098
:1027F000E4CF01F0E4CF00F01200D9CFE5FFE1CF44
:10280000D9FF00C0E5FF01C0E5FF02C0E5FF03C03E
:10281000E5FF04C0E5FF020EDBCF00F0030EDBCFC7
:1028200001F0040EDBCF02F00F01335111E182EC15
:1028300016F0036EF3CF04F003C0E5FF04C0F4FF0D
:1028400000C0E9FF01C0F3FF0250BAEC1AF016D045
:102850000F013351010A12E100C0E9FF01C0F3FF8B
:102860000250ECEC19F0006EF3CF01F00150E56E70
:102870000050E56E5AEC15F0E652E652E4CF04F053
:10288000E4CF03F0E4CF02F0E4CF01F0E4CF00F0B6
:10289000E4CFD9FF12000E0EF66E360EF76E000E64
:1028A000F86E0900F550056E0900F550066E04E15A
:1028B000056702D098EF14F00900F550006E09008A
:1028C000F550016E0900F550026E09000900F5503F
:1028D000E96E0900F550EA6E090009000900F5509B
:1028E000036E0900F550046E09000900F6CF07F0E9
:1028F000F7CF08F0F8CF09F000C0F6FF01C0F7FFEE
:1029000002C0F8FF035002E1045007E00900F5504F
:10291000EE6E0306F8E20406F9D707C0F6FF08C01A
:10292000F7FF09C0F8FF050601E2060657EF14F0AD
:10293000120000C0E5FF01C0E5FF02C0E5FFD0ECDA
:1029400017F0006ED0EC17F0016E0050026ED00E42
:102950000224006E0A0E005C05E30050026EF90EC0
:102960000224006E0150026ED00E0224016E0A0E87
:10297000015C05E30150026EF90E0224016E080E9F
:10298000005C12E2100E015CD8B00ED00038F00BE3
:102990000124006E48EC16F0016E015005E1005074
:1029A000E56E62EC19F0E652E4CF02F0E4CF01F0FC
:1029B000E4CF00F01200D9CFE5FFE1CFD9FF00C08E
:1029C000E5FF01C0E5FF02C0E5FF020ED924006E5D
:1029D000000EDA20016E800E026E030E0026000E3D
:1029E000012202220250E56E0150E56E0050E56EB4
:1029F000040EDBCFE5FF030EDBCFE5FF020EDBCFDE
:102A0000E5FF0F012C51E56E2B51E56E2A51E56E65
:102A10000EEC00F0006EF3CF01F0090EE12601C0CC
:102A2000F3FF0050E4CF02F0E4CF01F0E4CF00F078
:102A3000E4CFD9FF1200D9CFE5FFE1CFD9FF00C025
:102A4000E5FF01C0E5FF02C0E5FF03C0E5FF020EA0
:102A5000DBCF00F0030EDBCF01F0040EDBCF02F082
:102A60000F0133510DE1C0EC19F0036E03C0E5FF17
:102A700000C0E9FF01C0F3FF0250DDEC1AF00FD0F7
:102A80000F013351010A0BE100C0E9FF01C0F3FF60
:102A9000025051EC1AF0E56E21EC18F0E652E4CF4A
:102AA00003F0E4CF02F0E4CF01F0E4CF00F0E4CF94
:102AB000D9FF1200D9CFE5FFE1CFD9FF00C0E5FF74
:102AC00001C0E5FF02C0E5FF03C0E5FF020EDBCF5A
:102AD00000F0030EDBCF01F07EC402F07FC403F0F0
:102AE00004017E3F01D07F2B0150E56E0250E56E60
:102AF000FAEC17F0E652E6527EC402F07FC403F00F
:102B000004017E3F01D07F2B0050E56E0250E56E40
:102B1000FAEC17F0E652E652E4CF03F0E4CF02F00D
:102B2000E4CF01F0E4CF00F0E4CFD9FF1200D9CF19
:102B3000E5FFE1CFD9FF00C0E5FF01C0E5FF02C01E
:102B4000E5FF03C0E5FF04C0E5FF020EDBCF00F0A8
:102B500076C401F0026A014A022A77C403F0046ACB
:102B60000150031803E10250041801E001D00ED017
:102B7000000E04017625016E026A070E022201C0D2
:102B8000E9FF02C0EAFF00C0EFFF762BE4CF04F0BC
:102B9000E4CF03F0E4CF02F0E4CF01F0E4CF00F0A3
:102BA000E4CFD9FF1200D9CFE5FFE1CFD9FF00C0B4
:102BB000E5FF01C0E5FF02C0E5FF03C0E5FF020E2F
:102BC000DBCF00F0016AA0C402F0036A02500026C5
:102BD00003500122E56A800EE56E0150E56E00505B
:102BE000E56E77EC10F0006EF3CF01F0040EE126F5
:102BF000600E0026000E012200C0E9FF01C0EAFFBE
:102C0000EFCF00F00050E4CF03F0E4CF02F0E4CFC8
:102C100001F0E4CF00F0E4CFD9FF1200F3CFE5FFDD
:102C2000F4CFE5FFE9CFE5FFEACFE5FFFACFE5FF17
:102C3000FBCFE5FF040174510401366F04017551A7
:102C40000401376FD650346FD750356FF2A411D0CE
:102C50000401743F01D0752BF294040174510401F6
:102C6000366F040175510401376FD650346FD75059
:102C7000356F24EC1BF0E4CFFBFFE4CFFAFFE4CF89
:102C8000EAFFE4CFE9FFE4CFF4FFE4CFF3FF110064
:102C900000C0E5FF01C0E5FF02C0E5FF010E006EC8
:102CA000D0EC17F0016E01C002F0015023E000509B
:102CB000E56E82EC1AF0016EE652015010E10A0E48
:102CC000005C0BE20A0E006EE56E82EC1AF0016EFB
:102CD000E652015004E1E8680ED0E8680CD00150DB
:102CE000021802E0E86807D0002A1B0E005CD8E357
:102CF000E86801D0E86AE4CF02F0E4CF01F0E4CF65
:102D000000F0120000C0E5FF01C0E5FF02C0E5FFD2
:102D100003C0E5FF7EC400F07FC401F004017E3FE4
:102D200001D07F2B0050E56E82EC1AF0E652036E64
:102D3000026A7EC400F07FC401F004017E3F01D02E
:102D40007F2B0050E56E82EC1AF0E652016A021207
:102D50000150031203C0F3FF0250E4CF03F0E4CFAD
:102D600002F0E4CF01F0E4CF00F01200D9CFE5FF8C
:102D7000E1CFD9FF00C0E5FF01C0E5FF02C0E5FFDC
:102D800003C0E5FF020EDBCF00F0030EDBCF01F046
:102D9000040EDBCF02F00050020DF450036EF3CFAF
:102DA00000F0240E0026040E032200C0E9FF03C039
:102DB000EAFF01C0EEFF02C0EFFFE4CF03F0E4CF73
:102DC00002F0E4CF01F0E4CF00F0E4CFD9FF12002D
:102DD000D9CFE5FFE1CFD9FF00C0E5FF01C0E5FF96
:102DE00002C0E5FF03C0E5FF04C0E5FF020EDBCF34
:102DF00000F0030EDBCF01F0040EDBCF02F0050E76
:102E0000DBCF03F0060EDBCFE9FF070EDBCFEAFFD7
:102E1000080EDBCF04F040EC04F0E4CF04F0E4CF84
:102E200003F0E4CF02F0E4CF01F0E4CF00F0E4CF10
:102E3000D9FF120000C0E5FF01C0E5FF02C0E5FFB9
:102E4000006E390E04017B25016E026A040E022217
:102E500001C0E9FF02C0EAFF00C0EFFF220E7B5D68
:102E600001E27B2B00500A0A0FE104017B51E56E61
:102E7000800EE56E040EE56E390EE56EFCEC0FF08B
:102E8000040EE12604017B6BE4CF02F0E4CF01F0F5
:102E9000E4CF00F012000401766B0401776B0401AB
:102EA00078698B809490B06A3F0EAF6EB886AC8A1A
:102EB000AC84AC8CAC90AB8CAB8E0401976B0F01E7
:102EC000356B0401946B0401956B0401966B000E45
:102ED000E56A82EC1AF004017A6FE6529F989F9A95
:102EE000010E0401796F0F012A6B2B6B2F0E2C6FD3
:102EF00090EC1AF01200D9CFE5FFE1CFD9FF00C066
:102F0000E5FF01C0E5FF02C0E5FF03C0E5FF020EDB
:102F1000DBCF00F0030EDBCF01F0040EDBCF02F0BD
:102F2000050EDBCF03F0060EDBCFE9FF070EDBCF8C
:102F3000EAFFC1EC07F0E4CF03F0E4CF02F0E4CF06
:102F400001F0E4CF00F0E4CFD9FF12000401745186
:102F500004018C6F0401755104018D6FD6508A6F86
:102F6000D7508B6F8C510401741905E104018D5108
:102F7000040175190CE00401745104018C6F040103
:102F8000755104018D6FD6508A6FD7508B6F8DC4E9
:102F9000E9FF8CC4F4FF8BC4F3FF04018A511200D3
:102FA00000C0E5FF01C0E5FF0401955104019E1931
:102FB00005E0040195510401941902E1E86A15D075
:102FC00095C400F00401952B016A600E0026000EE6
:102FD000012200C0E9FF01C0EAFFEFCF00F09551E8
:102FE000800A02E10401956B0050E4CF01F0E4CFC8
:102FF00000F01200D9CFE5FFE1CFD9FF00C0E5FF17
:10300000020EDBCF00F0030EDBCFA8FF00C0A9FF4C
:10301000A69EA69CA684F29EF29C550EA76EAA0EB2
:10302000A76EA682A6A202D00000FCD7E86AA6B6C8
:10303000E82AA694F28EF28CE4CF00F0E4CFD9FF18
:103040001200D9CFE5FFE1CFD9FF00C0E5FF01C0F5
:10305000E5FF02C0E5FF020EDBCF00F07EC401F009
:103060007FC402F004017E3F01D07F2B0050E56E4B
:103070000150E56EFAEC17F0E652E652E4CF02F0AA
:10308000E4CF01F0E4CF00F0E4CFD9FF1200D8CFB5
:10309000E5FFE0CFE5FFE56EF3CFE5FFF4CFE5FF19
:1030A000E9CFE5FFEACFE5FFFACFE5FFFBCFE5FF8C
:1030B00029EC0AF0E4CFFBFFE4CFFAFFE4CFEAFF0C
:1030C000E4CFE9FFE4CFF4FFE4CFF3FFE450E4CF33
:1030D000E0FFE4CFD8FF100013EC1BF052EC11F02E
:1030E0008A9C939C400EE56E800EE56E0F0EE56E99
:1030F0008A0EE56E000EE56A86EC12F0050EE126FA
:103100008A9E939E800EE56EE56E0F0EE56E8A0E2A
:10311000E56E010EE56E86EC12F0050EE12612005A
:1031200000C0E5FF21EC1BF00401896B806B8983F3
:10313000006A89B3002A0050010BE844F46E805104
:10314000FD0BF410806FD58ED59CD59AD588D59679
:10315000D594D582D580F28AF184D08EF28EF28C0D
:10316000E4CF00F01200E8AE0AD0F3CFEAFFEE5051
:10317000EECFF3FFEECFF4FFEECFE9FF1200E8BC95
:1031800040EF1BF0E9CFF6FFF3CFF7FFF86E090031
:10319000F5500900F5CFF3FF0900F5CFF4FF090062
:1031A000F5CFE9FF120000C0E5FF01C0E5FF040113
:1031B00076510401771902E1E86A0FD0000E04018C
:1031C0007725006E016A070E012200C0E9FF01C0E9
:1031D000EAFFEFCF00F0772B0050E4CF01F0E4CF0F
:1031E00000F01200F2CFEAFFF29EA69EA69CA684F3
:1031F000E9CFA9FFF3CFAAFFE4CFA8FFE8EC1AF0CC
:10320000F4CFA8FFE8EC1AF0F6CFA8FFE8EC1AF02C
:10321000F7CFA8FFE8EC1AF0A694EABEF28E1200EF
:10322000F2CFF6FFF29EA69EA69CE9CFA9FFF3CFB0
:10323000AAFFA680A850A94AAA2AA680A8CFF3FF71
:10324000A94AAA2AA680A8CFF4FFA94AAA2AA6803A
:10325000A8CFEAFFF6BEF28E1200E8AE08D0F3CF98
:10326000EAFFEE50EECFF3FFEECFF4FF1200E8BC22
:1032700042EF1BF0E9CFF6FFF3CFF7FFF86E09003E
:10328000F5500900F5CFF3FF0900F5CFF4FF120068
:10329000F2CFEAFFF29EA69EA69CA684E9CFA9FFE4
:1032A000F3CFAAFFE4CFA8FFE8EC1AF0F4CFA8FF11
:1032B000E8EC1AF0F6CFA8FFE8EC1AF0A694EABE04
:1032C000F28E1200D9CFE5FFE1CFD9FF00C0E5FFB4
:1032D000020EDBCF00F000C07AF40050E56E000E65
:1032E000E56AFAEC17F0E652E652E4CF00F0E4CFDC
:1032F000D9FF1200F2CFF6FFF29EA69EA69CE9CF60
:10330000A9FFF3CFAAFFA680A850A94AAA2AA6809F
:10331000A8CFF3FFA94AAA2AA680A8CFF4FFF6BE39
:10332000F28E120000C0E5FF01C0E5FF600E04014F
:103330009525006E016A000E012200C0E9FF01C060
:10334000EAFFEFCF00F00050E4CF01F0E4CF00F04F
:103350001200D9CFE5FFE1CFD9FF00C0E5FF020E93
:10336000DBCF00F0610E005C05E37B0E005C02E247
:10337000010E01D0E86AE4CF00F0E4CFD9FF1200DB
:1033800000C0E5FF01C0E5FF7EC400F07FC401F08E
:1033900004017E3F01D07F2B0050E56E82EC1AF0D5
:1033A000E652E4CF01F0E4CF00F01200D9CFE5FF00
:1033B000E1CFD9FF00C0E5FF020EDBCF00F000C077
:1033C00079F4005004E190EC1AF09D9A9D98E4CFB6
:1033D00000F0E4CFD9FF1200E8AE06D0F3CFEAFF49
:1033E000EE50EECFF3FF1200E8BC3EEF1BF0E9CF4A
:1033F000F6FFF3CFF7FFF86E0900F5500900F5CF9F
:10340000F3FF1200F2CFEAFFF29EA69EA69CA684CE
:10341000E9CFA9FFF3CFAAFFE4CFA8FFE8EC1AF0A9
:10342000F4CFA8FFE8EC1AF0A694EABEF28E1200E0
:1034300018EEFFF028EEFFF0F86AA68EA69CE96869
:103440000E0EEA6E0068000EED6A0050FDE14BECD6
:1034500014F006EC00F0FFD7F2CFF6FFF29EA69E26
:10346000A69CE9CFA9FFF3CFAAFFA680A850A94A3E
:10347000AA2AA680A8CFF3FFF6BEF28E1200F2CFE2
:10348000EAFFF29EA69EA69CA684E9CFA9FFF3CFF1
:10349000AAFFE4CFA8FFE8EC1AF0A694EABEF28EE9
:1034A0001200E8AE04D0F3CFEAFFEE501200E8BC01
:1034B0003CEF1BF0E9CFF6FFF3CFF7FFF86E090002
:1034C000F5501200E8AE0BD0F3CFEAFFE4CFEEFFE9
:1034D000F4CFEEFFF6CFEEFFF7CFEEFF1200E8BC21
:1034E0003AEF1BF01200E8AE09D0F3CFEAFFE4CFC9
:1034F000EEFFF4CFEEFFF6CFEEFF1200E8BC44EF94
:103500001BF01200D9CFE5FFE1CFD9FF020EDBCFD0
:10351000A9FFA69CA69EA680A850E4CFD9FF1200C2
:10352000ACA2FED78B80AE500000AE50AB98AB88FB
:10353000AB869D8A9D981200256420007EA20BD048
:103540000F012751E96E2851EA6E0401A11DEF1603
:103550000F014E917E921200F2CFF6FFF29EA69ED0
:10356000A69CE9CFA9FFF3CFAAFFA680A850F6BE7C
:10357000F28E1200E8AE07D0F3CFEAFFE4CFEEFF01
:10358000F4CFEEFF1200E8BC38EF1BF01200700E13
:10359000D36E9B8CFF0E9268936894689668626AFB
:1035A000F19E120000C0E5FF48EC16F0006E0050DE
:1035B00001E1FF00E4CF00F01200E8AE05D0F3CF48
:1035C000EAFFE4CFEEFF1200E8BC36EF1BF012007A
:1035D000550EA76EAA0EA76EA682A6B2FED7A94A5E
:1035E000AA2A010E0F01336F1C0E04017E6F7F6B40
:1035F0001200D0EC17F0140A02E120EC12F01200D5
:103600000F01336B1C0E04017E6F7F6B12000100F3
:1036100030360000740400000A00000060EC0EF078
:1036200007EC0CF0120090EC18F04BEC17F01200C5
:1036300000000000FF0000000000ACA2FED7AD6E4D
:103640001200C7EC1AF012009EEC1AF012000401EE
:103650009551120004019F5112000401795112008A
:1036600004017C6B1200E8CF7FFF12003FEF1AF0DD
:1036700002EF1AF0F2EF18F0ACEF1AF02CEF1AF09C
:0C36800010EF19F07AEF19F048EF19F084
:00000001FF
